:06000000020033020E664F
:03000B00020E677B
:03001300020E8159
:03001B00020E8250
:03002300020E8347
:03002B00020E843E
:10003300759840758780758921758DFF758BFF7560
:100043008850D299758160758CFA758A0075A8827B
:1000530075900075B0FF7535FF7537FF7539FF75FE
:100063003BFF753DFF753FFF7541FF7543FF7545C9
:10007300FF753600753800753A00753C00753E0013
:1000830075400075420075440075300C753100D21F
:10009300A0D2A1782076FF08B830FAC2A27E80DF12
:1000A300FEDEFCC280C287C286D285D284D2A3C2BE
:1000B300A3DFFEDFFEDFFEDFFEDFFED2A3C2A3DF90
:1000C300FED2A3C2A3DFFEC284D2A3C2A3742812AA
:1000D3001088DFFE7408121088DFFE740612108881
:1000E300DFFE7410121088DFFE740C121088DFFE1E
:1000F3007401121088DFFEDFFE74401210887F4007
:10010300901321E4931210ADA3DFF87480121088CA
:100113007F14901361E4931210ADA3DFF874C0123F
:1001230010887F14901375E4931210ADA3DFF8DFEA
:10013300FEDEFCDFFEDEFCDFFEDEFCDFFEDEFC744B
:10014300801210887F14901389E4931210ADA3DFFB
:10015300F874C01210887F1490139DE4931210ADAD
:10016300A3DFF8759000D2A0D2A17880E670257540
:10017300B0FE75A00120A00F300019C200760890D0
:100183001195120F25800D20000AD20076089011D8
:1001930098120F257881E6702575B0FE75A00220B0
:1001A300A10F300119C201760890119B120F25800F
:1001B3000D20010AD201760890119E120F25789026
:1001C300E6702575B0FB75A00120A00F301019C291
:1001D3001076089011A1120F25800D20100AD2105D
:1001E30076089011A4120F257891E6702575B0FB5F
:1001F30075A00220A10F301119C21176089011A722
:10020300120F25800D20110AD21176089011AA121F
:100213000F257898E6702575B0F775A00120A00F1B
:10022300301819C21876089011AD120F25800D20D1
:10023300180AD21876089011B0120F257899E67033
:100243002575B0F775A00220A10F301919C21976D0
:10025300089011B3120F45800D20190AD2197608A0
:100263009011B6120F4578A0E6702575B0EF75A012
:100273000120A00F302019C22076089011B9120F67
:1002830025800D20200AD22076089011BC120F255C
:1002930075B0EF75A00220A126753207120E9312D6
:1002A3000E85D53206753201120E93120E8C75B07F
:1002B300EF75A00220A10820190302115E80E378E4
:1002C300A8E6702575B0DF75A00120A00F302819AE
:1002D300C22876089011BF120F25800D20280AD25C
:1002E3002876089011C2120F2575B0DF75A0022081
:1002F300A126753207120EB8120E85D53206753255
:1003030001120EB8120E8C75B0DF75A00220A10881
:1003130020190302115E80E378B0E6702575B0BF43
:1003230075A00120A00F303019C23076089011C596
:10033300120F25800D20300AD23076089011C81292
:100343000F2575B0BF75A00220A120753207120ECC
:10035300DD120E85D53206753201120EDD120E8CBA
:1003630075B0BF75A00220A10280E978B8E67025B8
:1003730075B07F75A00120A00F303819C2387608F8
:100383009011CB120F25800D20380AD238760890B1
:1003930011CE120F2575B07F75A00220A1207532F2
:1003A30007120F01120E85D53206753201120F01A5
:1003B300120E8C75B07F75A00220A10280E97590A2
:1003C300FFC2A0C2A178C0E6702575B0FE7590018A
:1003D30020900F304019C24076089011D1120F259A
:1003E300800D20400AD24076089011D4120F257850
:1003F300C1E6702575B0FE75900220910F3041194A
:10040300C24176089011D7120F25800D20410AD2E0
:100413004176089011DA120F2578C2E6702575B07F
:10042300FE75900420920F304219C2427608901153
:10043300DD120F25800D20420AD24276089011E08A
:10044300120F2578C3E6702575B0FE7590082093CA
:100453000F304319C24376089011E3120F25800D24
:1004630020430AD24376089011E6120F2578C4E69A
:10047300702575B0FE75901020940F304419C24456
:1004830076089011E9120F25800D20440AD2447694
:10049300089011EC120F2578C5E6702575B0FE752E
:1004A300902020950F304519C24576089011EF1220
:1004B3000F25800D20450AD24576089011F2120FC0
:1004C3002578C6E6702575B0FE75904020960F30EE
:1004D3004619C24676089011F5120F25800D204665
:1004E3000AD24676089011F8120F2578C7E67025D0
:1004F30075B0FE75908020970F304719C247760874
:100503009011FB120F25800D20470AD247760890E1
:1005130011FE120F2578D0E6702575B0FB7590019A
:1005230020900F305019C2507608901201120F25F7
:10053300800D20500AD2507608901204120F2578AD
:10054300D1E6702575B0FB75900220910F305119DB
:10055300C2517608901207120F25800D20510AD23E
:1005630051760890120A120F2578D2E6702575B0DD
:10057300FB75900420920F305219C25276089012E4
:100583000D120F25800D20520AD2527608901210B8
:10059300120F2578D3E6702575B0FB75900820936C
:1005A3000F305319C2537608901213120F25800D82
:1005B30020530AD2537608901216120F2578D4E6E8
:1005C300702575B0FB75901020940F305419C254E8
:1005D3007608901219120F25800D20540AD25476F2
:1005E3000890121C120F2578D5E6702575B0FB759F
:1005F300902020950F305519C255760890121F127E
:100603000F25800D20550AD2557608901222120F1D
:100613002578D6E6702575B0FB75904020960F308F
:100623005619C2567608901225120F25800D2056B2
:100633000AD2567608901228120F2578D7E670252D
:1006430075B0FB75908020970F305719C257760805
:1006530090122B120F25800D20570AD2577608903F
:10066300122E120F2578D8E6702575B0F775900114
:1006730020900F305819C2587608901231120F2566
:10068300800D20580AD2587608901234120F25781C
:10069300D9E6702575B0F775900220910F3059197E
:1006A300C2597608901237120F25800D20590AD2AD
:1006B30059760890123A120F2578DAE6702575B04C
:1006C300F775900420920F305A19C25A7608901287
:1006D3003D120F25800D205A0AD25A7608901240F7
:1006E300120F2578DBE6702575B0F7759008209317
:1006F3000F305B19C25B7608901243120F25800DF1
:10070300205B0AD25B7608901246120F2578DCE64E
:10071300702575B0F775901020940F305C19C25C8A
:100723007608901249120F25800D205C0AD25C7660
:100733000890124C120F2578DDE6702575B0F77519
:10074300902020950F305D19C25D760890124F12EC
:100753000F25800D205D0AD25D7608901252120F8C
:100763002578DEE6702575B0F775904020960F303A
:100773005E19C25E7608901255120F25800D205E19
:100783000AD25E7608901258120F2578DFE670259C
:1007930075B0F775908020970F305F19C25F7608A8
:1007A30090125B120F25800D205F0AD25F760890AE
:1007B300125E120F2578E0E6702575B0EF75900193
:1007C30020900F306019C2607608901261120F25D5
:1007D300800D20600AD2607608901264120F25788B
:1007E300E1E6702575B0EF75900220910F30611925
:1007F300C2617608901267120F25800D20610AD21C
:1008030061760890126A120F2578E2E6702575B0BA
:10081300EF75900420920F306219C262760890122D
:100823006D120F25800D20620AD262760890127035
:10083300120F2578E3E6702575B0EF7590082093C5
:100843000F306319C2637608901273120F25800D5F
:1008530020630AD2637608901276120F2578E4E6B5
:10086300702575B0EF75901020940F306419C26431
:100873007608901279120F25800D20640AD26476CF
:100883000890127C120F2578E5E6702575B0EF7598
:10089300902020950F306519C265760890127F125B
:1008A3000F25800D20650AD2657608901282120FFB
:1008B3002578E6E6702575B0EF75904020960F30E9
:1008C3006619C2667608901285120F25800D206680
:1008D3000AD2667608901288120F2578E7E670250B
:1008E30075B0EF75908020970F306719C26776084F
:1008F30090128B120F25800D20670AD2677608901D
:10090300128E120F2578E8E6702575B0DF75900119
:1009130020900F306819C2687608901291120F2543
:10092300800D20680AD2687608901294120F2578F9
:10093300E9E6702575B0DF75900220910F306919D3
:10094300C2697608901297120F25800D20690AD28A
:1009530069760890129A120F2578EAE6702575B029
:10096300DF75900420920F306A19C26A76089012DC
:100973009D120F25800D206A0AD26A76089012A074
:10098300120F2578EBE6702575B0DF75900820937C
:100993000F306B19C26B76089012A3120F25800DCE
:1009A300206B0AD26B76089012A6120F2578ECE61C
:1009B300702575B0DF75901020940F306C19C26CE0
:1009C30076089012A9120F25800D206C0AD26C763E
:1009D300089012AC120F2578EDE6702575B0DF751F
:1009E300902020950F306D19C26D76089012AF12CA
:1009F3000F25800D206D0AD26D76089012B2120F6A
:100A03002578EEE6702575B0DF75904020960F309F
:100A13006E19C26E76089012B5120F25800D206EE6
:100A23000AD26E76089012B8120F2578EFE6702579
:100A330075B0DF75908020970F306F19C26F7608FD
:100A43009012BB120F25800D206F0AD26F7608908B
:100A530012BE120F2578F0E6702575B0BF759001B0
:100A630020900F307019C27076089012C1120F25B2
:100A7300800D20700AD27076089012C4120F257868
:100A8300F1E6702575B0BF75900220910F30711992
:100A9300C27176089012C7120F25800D20710AD2F9
:100AA3007176089012CA120F2578F2E6702575B098
:100AB300BF75900420920F307219C272760890129B
:100AC300CD120F25800D20720AD27276089012D0B3
:100AD300120F2578F3E6702575B0BF759008209343
:100AE3000F307319C27376089012D3120F25800D3D
:100AF30020730AD27376089012D6120F2578F4E683
:100B0300702575B0BF75901020940F307419C2749E
:100B130076089012D9120F25800D20740AD27476AC
:100B2300089012DC120F2578F5E6702575B0BF75B5
:100B3300902020950F307519C27576089012DF1238
:100B43000F25800D20750AD27576089012E2120FD8
:100B53002578F6E6702575B0BF75904020960F3066
:100B63007619C27676089012E5120F25800D20764D
:100B73000AD27676089012E8120F2578F7E67025E8
:100B830075B0BF75908020970F307719C2777608BC
:100B93009012EB120F25800D20770AD277760890FA
:100BA30012EE120F2578F8E6702575B07F75900167
:100BB30020900F307819C27876089012F1120F2521
:100BC300800D20780AD27876089012F4120F2578D7
:100BD300F9E6702575B07F75900220910F30791971
:100BE300C27976089012F7120F25800D20790AD268
:100BF3007976089012FA120F2578FAE6702575B007
:100C03007F75900420920F307A19C27A7608901279
:100C1300FD120F25800D207A0AD27A7608901300F0
:100C2300120F2578FBE6702575B07F759008209329
:100C33000F307B19C27B7608901303120F25800DAA
:100C4300207B0AD27B7608901306120F2578FCE6E8
:100C5300702575B07F75901020940F307C19C27C7D
:100C63007608901309120F25800D207C0AD27C761A
:100C73000890130C120F2578FDE6702575B07F756B
:100C8300902020950F307D19C27D760890130F12A6
:100C93000F25800D207D0AD27D7608901312120F46
:100CA3002578FEE6702575B07F75904020960F304D
:100CB3007E19C27E7608901315120F25800D207EB3
:100CC3000AD27E7608901318120F2578FFE6702556
:100CD30075B07F75908020970F307F19C27F76089B
:100CE30090131B120F25800D207F0AD27F76089068
:100CF300131E120F257590FFD2A0D2A17580FFD2CB
:100D0300A27407B535037535FF0535E535A2E092C5
:100D1300A4A2E192A5A2E292A6C2AFD2A7C2A7E47F
:100D2300B53503020D5604B53503020D7704B53509
:100D330003020D9804B53503020DB904B53503025A
:100D43000DDA04B53503020DFB04B53503020E1CA1
:100D5300020E3DE580F536A837A936120F6340062B
:100D630024FE500D8005120F685006853637120F8A
:100D73006F020E5EE580F538A839A938120F63407B
:100D83000624FE500D8005120F685006853839126F
:100D93000F93020E5EE580F53AA83BA93A120F6362
:100DA300400624FE500D8005120F685006853A3B1D
:100DB300120FB7020E5EE580F53CA83DA93C120F69
:100DC30063400624FE500D8005120F685006853CD3
:100DD3003D120FDB020E5EE580F53EA83FA93E12F1
:100DE3000F63400624FE500D8005120F68500685E0
:100DF3003E3F120FFF020E5EE580F540A841A94079
:100E0300120F63400624FE500D8005120F68500632
:100E1300854041121023020E5EE580F542A843A9E6
:100E230042120F63400624FE500D8005120F6850D6
:100E330006854243121047020E5EE580F544A8453D
:100E4300A944120F63400624FE500D8005120F685B
:100E53005006854445121064020E5ED2AF0201664D
:100E630002003332C0D0C0E0C0007880E6600116D3
:100E730008B800F8758CFAD000D0E0D0D032323206
:100E830032327E20DFFEDEFC227E60DFFEDEFC22CD
:100E9300748012108805307419B53003753000E57D
:100EA300307F049013B1E5302323931210ADA3DFF9
:100EB300F512117C227480121088153074FFB5303E
:100EC30003753018E5307F049013B1E53023239385
:100ED3001210ADA3DFF512117C223099FDC2997572
:100EE30099C074C01210883099FDC299053174807D
:100EF300B53103753100E531F5991210FE223099B1
:100F0300FDC2997599C074C01210883099FDC299B9
:100F1300153174FFB5310375317FE531F599121041
:100F2300FE22E4933099FDC299F599A3E493253009
:100F33003099FDC299F599A3E4933099FDC299F5CF
:100F43009922E4933099FDC299F599A3E4933099DA
:100F5300FDC299F599A3E4933099FDC299F59922BD
:100F6300C2D7E89922C2D7E99824FE223099FDC25C
:100F7300997599E074D11210883099FDC2997599C9
:100F8300003099FDC299E536C313F5991210FE227C
:100F93003099FDC2997599B0748D1210883099FDFE
:100FA300C29975990B3099FDC299E538C313F59928
:100FB3001210FE223099FDC2997599B074891210EE
:100FC300883099FDC29975990A3099FDC299E53A1D
:100FD300C313F5991210FE223099FDC2997599B089
:100FE30074851210883099FDC2997599073099FD5F
:100FF300C299E53CC313F5991210FE223099FDC244
:10100300997599B074C91210883099FDC299759970
:10101300053099FDC299E53EC313F5991210FE22DE
:101023003099FDC2997599B074C51210883099FD35
:10103300C2997599013099FDC299E540C313F59999
:101043001210FE223099FDC2997599D07491121035
:10105300883099FDC299E542C313F5991210FE2217
:10106300223099FDC2997599B074CD1210883099C8
:10107300FDC2997599023099FDC299E544C313F5F0
:10108300991210FE22C2A2C2803392873392863312
:101093009285339284D2A3C2A33392873392863349
:1010A3009285339284D2A3C2A322C2A2D280339266
:1010B30087339286339285339284D2A3C2A3339229
:1010C30087339286339285339284D2A3C2A3227547
:1010D300F0648424301210AD740AC5F084243012F5
:1010E30010ADE5F024301210AD2275F00A842430DF
:1010F3001210ADC5F024301210AD22D2D575F064B4
:10110300847004C2D574F024301210AD740AC5F093
:1011130084700520D50274F024301210ADE5F0245C
:10112300301210AD2275F00A84700274F02430126C
:1011330010ADE5F024301210AD22E493A3B45E01A8
:10114300221210AD02113D70047420800AC313C330
:1011530013C313C313C3131210AD2212117C30999E
:10116300FDC2997599B03099FDC2997599783099F6
:10117300FDC2997599000200333099FDC2997599A2
:10118300B03099FDC29975997B3099FDC2997599D3
:101193000022905040805000905140805100905266
:1011A300408052009053408053009054408054003C
:1011B300B0407FB04000905540805500905640802D
:1011C3005600905740805700905840805800901820
:1011D30040801800901940801900901A40801A002E
:1011E300901B40801B00901C40801C00901D408081
:1011F3001D00901E40801E00901F40801F00902005
:1012030040802000902140802100902240802200D5
:101213009023408023009024408024009025408028
:1012230025009026408026009027408027009028A4
:1012330040802800902940802900902A40802A007D
:10124300902B40802B00902C40802C00902D4080D0
:101253002D00902E40802E00902F40802F00903044
:101263004080300090314080310090324080320025
:101273009033408033009034408034009035408078
:1012830035009036408036009037408037009038E4
:1012930040803800903940803900903A40803A00CD
:1012A300903B40803B00903C40803C00903D408020
:1012B3003D00903E40803E00903F40803F00904084
:1012C3004080400090414080410090424080420075
:1012D30090434080430090444080440090454080C8
:1012E3004500904640804600904740804700904824
:1012F30040804800904940804900904A40804A001D
:10130300904B40804B00904C40804C00904D40806F
:101313004D00904E40804E00904F40804F000000A3
:1013230000000000001F0000000000001F1F00005D
:101333000000001F1F1F000000001F1F1F1F0000D1
:10134300001F1F1F1F1F00001F1F1F1F1F1F001F26
:101353001F1F1F1F1F1F1F1F1F1F1F1F1F1F4D7516
:101363007A796B616E7420372076312E30622020BB
:10137300202020736D69616C656B2E7072762E7000
:101383006C202020202020432020203132372031A0
:10139300323720313237203132372020302020318C
:1013A30032372031323720313237203132372D4333
:1013B30020202D4465732D4420202D4573202D4579
:1013C30020202D4620202D4765732D4720202D41B9
:1013D30073202D4120202D4220202D482020204302
:1013E30020202B4369732B4420202B4469732B4506
:1013F30020202B4620202B4669732B4720202B4788
:1014030069732B4120202B4169732B4820202B43E8
:101413002020204D757A796B616E742037207631E8
:101423002E306220323030372D30372D30342028A3
:1014330063294164616D20536D69616C656B206A3A
:10144300616E6B6F6D757A796B616E744077702E18
:10145300706C207777772E736D69616C656B2E7076
:1014630072762E706C2057737A656C6B6965207089
:1014730072617761207A617374727A657A6F6E65CF
:101483002E204A616B69656B6F6C7769656B207A97
:101493006173746F736F77616E6961206B6F6D65D4
:1014A3007263796A6E65206B6F6475206E6965641B
:1014B3006F7A776F6C6F6E652E20416C6C2052696A
:1014C300676874732052657365727665642E20466F
:1014D30072656520666F72206E6F6E20636F6D6D2F
:0D14E30065726369616C206F6E6C792E205C
:00000001FF
